:020000040000FA
:1000000020288207FE34CD34993466344D343E3492
:10001000303422341A3413340D34093406340434A1
:100020000234013432082B02031D182831082A0239
:1000300008002B083402031D1F282A083302080079
:10004000F520C420CD20B7202A20272021280C1CF1
:1000500027280800B501B601003803193D282C18DF
:100060003428AC185D2843289420A120FF30AD002F
:100070000130AE00AC012C140800B601B5012C18FB
:100080004B28AC18542894202B08AE002A08AD0049
:10009000AC012C15080094201220031843281920C5
:1000A0000318432836280800942082209020371C0B
:1000B0005B28632008007420080094208220902090
:1000C0003714632008003608BA070318B90A391D27
:1000D0006F280330AE00FF30AD003710080039083C
:1000E000AE003A08AD00080036083A02AD00390803
:1000F000031CFF3EAE00AE1F08000030AE00AD0096
:1001000037140800AA0CAA0CAA0CAA0CAA0CAA0C58
:100110000330AA05AB0DAB0D0C302B052A040800EB
:100120000120B600B50108008B309F009F1896286B
:1001300083161E088312AA00AD001E08AB00AE0095
:1001400008000301B100B200B300B4002A080A3E5F
:10015000B1002B080318013EB2000A302A02B30096
:100160002B08031CFF3EB4000030B4020800851DBC
:10017000BC28851CC1280034AC012C14FF34B60106
:10018000B501AC01AC14FF3405143B308F00BB301B
:100190008E00013090000C100800E2202E08B900FB
:1001A0002D08BA000301AD040319D828AD0BD628D9
:1001B0000301AE040319E028AD0BDC28AE03D828F8
:1001C000051008000330A100D230A000A00BE628E3
:1001D000A10BE62808000430A000A00BED280000C9
:1001E00000000000000000000800831285010730B5
:1001F0009900831624309F003E3085008312893099
:100200009F002C10AC102C159420B601B5010130C4
:04021000B80008002A
:02400E00923FDF
:00000001FF
